:1074000080E189BD82E189BD09B400FEFDCF089508
:10741000CED569F08091E9008F931092E900A3D452
:1074200083FF01C022D58F9187708093E900089572
:107430008EEF0090E10008220092E1000895F20131
:10744000F999FECFF2BDE1BD0895F9DFF89A80B554
:1074500008C0F5DF1FBA80BD0FB6F894FA9AF99A02
:107460000FBE31962F010895E0E0F0E085919491F0
:107470000196089580EE8BB98BEA37D0109289007F
:107480008AEF8093880082E080936F0083E080938E
:1074900081004AD049D05C98EDE6F7E785913AD073
:1074A000E038E1F781E08093D7008AE482BF109250
:1074B000D8001092E2001092DA001092E10080E809
:1074C00008D019BC1EBA1092E00063D489E054D4ED
:1074D00081E98093D8000895A3E6B1E090E81AD03E
:1074E0008D939A95E1F7089586E008D010C083E067
:1074F00005D08F2F0FD08E2F0DD080E05E9A599837
:1075000009C005D085E0FADF05D080FDFDCF599A8E
:107510005E9808958EBD8DB587FFFDCF8EB5089519
:107520008FE08221E9F7F3DFE3E6F6E05C9A40E4DE
:1075300058E06081718198E08FEF60FF8F7070FF7D
:10754000807FE8DF669576959A95B1F7E058FF4F12
:107550005A9579F7EE5FF3404A9551F70895E3E6BF
:10756000F1E097FC38C094FC4FC092FE08958684E9
:10757000882011F4992459C0F894C089D78520E057
:1075800030E080E090E4AFEFBFEF119688199040B3
:10759000E0F72D01BD4F8D0127FD13C0E0E0F8E0BD
:1075A00011928EE7819392E4E11791939AE508F0A6
:1075B00092E4E334C9F781931082B5DFFE0121968E
:1075C00096DF8ADFF901F6D420583F4F040D151DD0
:1075D0008A9411F709C28301282D60906C01709084
:1075E0006B0141D019F48823C1F70895380188242C
:1075F0003AD0B9F580916A01821709F4830160904D
:107600006E0170906D01F4CF60906E0170906D010D
:107610002AD059F48823C1F708959FEF95FC03C041
:1076200096FE089591E097FB890E662477248301E6
:10763000222719D0B1F48823A1F380916A0136F092
:10764000881650F4821730F0213003C0881520F4DA
:10765000281710F48301282F60906E0170906D013F
:10766000E8CF3801822EF30142DF36DFC3E6D1E0F6
:10767000E6E6F7E709908591081621F4ED36D1F793
:107680000880801044CFC9E029DFCA95E9F7D0E12E
:1076900095FC1EC097FC53C094FC35C0C3E6D2E0F5
:1076A000E3E6F6E098E088E78E0F00840192E817A1
:1076B000E1F7884F09900192E817E1F7C858DF4FCA
:1076C0009A9589F72DDFC85FD340C33E49F749C07B
:1076D000C3E6D6E0EBE5FAE098E08E2F88570290FB
:1076E0000086E817E1F738960A900292E817E1F76A
:1076F0003897C857D0409A9581F712DFC850DC4FB1
:10770000C33E41F72EC0A3EEB6E0E3E6F6E09AE012
:10771000C6E00D9080818025807F802582958193B1
:10772000A336B90709F4B2E0E336F90709F4F2E049
:10773000E336FC0771F7F4DEDA9529F712C0A3EE01
:10774000B9E0E3E6FAE092E00E90829180258F7036
:10775000802582958083E336F907B1F7E1DEDA957B
:1077600071F78827089541524455424F5915003FFB
:1077700075205FA055A100A200A87F81CFB121AFE5
:107780000000FFFFCFCFFFFFFFFFCFCFFFFF0000C5
:10779000FE067E7E06FE46565616FE0656461EFE21
:1077A0003F61E9E3FFE3EBE3FFE3EBE3FFE16B3F83
:1077B0001201100102000008412336000100000000
:1077C000000109023E0002010080320904000001AC
:1077D000020201000524001001042402040524060D
:1077E0000001070582030800FF09040100020A00E6
:1077F00000000705040210000107058302100001C4
:1078000011241FBE04B714BE88E18093600010925B
:1078100060008EEF9AE09EBF8DBF222433242101A9
:107820004394310141018AC00F928F939F931F921D
:107830000FB60F9211244F936F938091DA0080FF5F
:1078400037C023C00F920FB68F939F93EF93FF9390
:1078500088278093850080938400E0E5F1E09281A1
:10786000907261F490818917980B908309F45D9A66
:1078700091818917980B918309F4289A239411F424
:107880008315381EFF91EF9154C08091D80080FF7E
:107890000FC08091DA008E7F8093DA008091D9004A
:1078A00080FF04C0ADDD81E08EBB02C019BC1EBAF2
:1078B0008091E10080FF0BC059D280FF08C059D2EF
:1078C0008091D800806205DE19BC85E08EBB809176
:1078D000E10084FF1AC04AD284FF17C091DD809175
:1078E000D8008F7DF6DD8FEEA4DD40D28F7E8160E3
:1078F00043D280915301882331F48091E30087FDC6
:1079000002C081E001C084E08EBB8091E10083FF72
:107910000CC02CD283FF09C087EF8BDD82E08EBBC9
:107920001092530185DD25D234D26F914F910F9083
:107930001F909F918F910FBE0F90189580E88093B4
:10794000610010926100B1E0B5BF82E085BF81EFB8
:1079500085B987EE84B91DB8769A10BA80EF81BBDD
:1079600082E68BB982EF8AB980E58CBDBDBDA0E00F
:10797000E0EBF7E705900D92A035E1F71D92BB30E3
:10798000E9F701FD09C000FF07C07C9B05C05DDD74
:10799000882312F069DD41F56DDD789464DE71F0C5
:1079A000ABE9B7E0E0E8F7E790E105900D929A9532
:1079B000E1F7A059BF4FE03BB9F7B6DD52D028DD63
:1079C00080915201807861F48FB18095807F6699B3
:1079D0001C9B8460982E21DE8110C1DD92FC02C0C8
:1079E000332062F741DD51F3F89489EB7EDD81E0CD
:1079F0008093E00010926F00109281001092850039
:107A00001092840081E085BF15BE2E9A2F9A2D9A80
:107A10005D9A289A0C940000A4D107C057D102C0E7
:107A2000C6D239F0A0D182FFFBCF85FFF7CF80917E
:107A3000F1000895082E83E095D185FD07C08AD115
:107A400002C0B5D269F08FD180FFFBCF0092F10068
:107A500080915201807221F45D9884E680935001F8
:107A600008957FD182FF34C180915201807221F448
:107A7000289884E680935101CFDF182F853431F4A4
:107A800022248EE7382EDBDC8DE00BC1843511F427
:107A9000C3DFFACF8C34C1F38035B1F3843721F4DE
:107AA00084E4C8DF80E0FDC0813611F489E5F9C0C7
:107AB000813429F4B1DF582EAFDF482EE5CF80376F
:107AC00011F483E5EEC0833539F4E6E6F7E78591F6
:107AD000B1DFED36E1F7E6C0863521F481E3AADFB8
:107AE00086E3DFC0863761F481E3669B8E5F1C9B73
:107AF0008F5FA0DF8FB1809582958F708F5BD1C033
:107B00008837A9F489DF80935201289A84FD289848
:107B10005D9A83FD5D982E9A81FD2E982F9A82FDA5
:107B20002F982D9A80FD2D9887FD8824ADCF8A3619
:107B300049F48FE9E3DCC3E0EDDC7CDFCA95E1F7D3
:107B4000E6DCB0C0833731F487E874DF85E972DFA3
:107B50008EE1A7C0853639F4E0E8F3E73ED2E0587D
:107B6000F040E0F791CF823631F489E563DF80E0C1
:107B700061DF80E896C0823419F0873609F07DC055
:107B800033244ADFD82F48DFC82F46DF082F83541D
:107B9000843008F085C0063411F4440C551CF20101
:107BA00010926F001736B9F4033489F483E0A0DC37
:107BB000B1DC8EB51EBC3EDF0DB42197D1F7A7DC3A
:107BC00008C0063411F4859101C03FDC33DF2197F2
:107BD000C2F72F014AC00334A9F4E11104C084DCC8
:107BE00088ED86DC8EDC80DC82E082DC15DF0DB483
:107BF0008EBDCA95D9F731968EDC83DCDA9569F7AC
:107C00002F0131C00634F1F49F01F437D8F4E5D1E7
:107C100019C002DF063461F4C0FB46F0F43728F4E3
:107C2000182E81E087BFE89511243296082E0AC0ED
:107C3000043439F4DF01B370AD59B94F8D933196E7
:107C400001C007DC21972AF7043431F42F01F370C7
:107C5000FE2B49F469DC07C0063429F42F01F90131
:107C6000F43708F4B8D18DE0E5DE063411F456940B
:107C7000479482E080936F0015C08237E1E049F0BD
:107C80008634E0E031F08E34E3E019F0813531F4F0
:107C9000E2E0F0E089E087BF849103C08B3111F00E
:107CA0008FE3C8DE83E0C1DB55D095FF03C009C078
:107CB0007ED171F058D080FFFBCF4CD002C077D17D
:107CC00039F051D080FFFBCF84E0AFDB8BE743C0BE
:107CD0000895E4E5F1E067E090915B0180915C013B
:107CE000913231F0913AE1F58132D1F55ED181C026
:107CF000823271F48191805B8191844089F5809119
:107D00005D0180FD2DC0F89481E08093E00078CD86
:107D1000803231F54AD14BD1E9F08530D9F023D00A
:107D200083FD18C082FFF7CF04C081DE81936150CC
:107D300031F09091F3008091F200892BB1F7C6DF0A
:107D4000611549F704C033D129F0853019F00BD003
:107D500080FFF9CF8EE79091E80089238093E800B7
:107D6000089584E062DB8091E80008958091E2004C
:107D70000895FCDF8E7F80618093E200089582E0A9
:107D800061EC09D083E061E802D084E060E842E180
:107D900003C080E060E042E048DB81E007D0109261
:107DA000ED006093EC004093ED0008959091EB009E
:107DB000892B8093EB00089560E0923029F0913098
:107DC00029F4E0E062E102C0E2E16EE3F1E008954F
:107DD00080915B0188234CF402C0E9D0C1F3C3DF7A
:107DE00082FFFBCF73CFE3D091F3BDDF80FFFBCFEA
:107DF000B1CF40916101509162014617510520F0C9
:107E0000462F611509F4A6DF50E022C0D0D061F101
:107E1000853051F1A8DF83FD59CFA5DF82FD21C058
:107E200080FF16C03091F3002091F20006C08191CE
:107E30008093F10041502F5F3F4F411519F02830DA
:107E40003105A8F350E02830310509F451E082DF14
:107E50004115E1F65523D1F604C0A9D029F08530AB
:107E600019F081DF82FFF9CF31CFEBE5F1E0DFDD03
:107E70008193E336E1F72DDF76DF83FF91C08091B8
:107E80005B0190915C01913009F170F09330F1F059
:107E9000953009F444C0963009F456C0983009F47E
:107EA00060C0993059F767C0823841F780915F010F
:107EB000BBDA2091EB001092E90077D0229526954D
:107EC00021702093F1001092F10052C0882311F02C
:107ED0008230A1F68F71823089F680915D0188230E
:107EE000D1F420915F01277049F22093E90080913D
:107EF000EB0080FF10C0933011F480E20BC080E1F2
:107F000055DF81E0880F2A95E9F78093EA00109207
:107F1000EA0088E04BDF1092E90047D02AC08823AE
:107F200091F410915D0110680FB7F8943ED050DFC6
:107F30001ADF80FFFDCF1093E300103883E009F4CF
:107F400082E08EBB0FBF2CC08058823048F58091F4
:107F50005D0190915E0130DF603011F126D049DF84
:107F60001FC08038E9F421D0809153018093F10043
:107F7000F1DE2EDF15C0882399F490915D019230D7
:107F800078F49093530111D023DF8091530188231B
:107F900021F48091E30091E087FD94E09EBBEFDE49
:107FA000E2DE83FF089580E201DF87EFD4CE8EB357
:107FB00088230895A3E6B1E0F437B8F40ED090E436
:107FC0000D901D9081E087BFE89532969A95C1F794
:107FD0001124E058F04085E001C083E001D081E148
:0C7FE00087BFE89507B600FCFDCF0895B0
:067FFA003136DDCFFBDC97
:040000030000740085
:00000001FF
